:10000000AEC0FECFFDCFFCCFFBCFFACFF9CFF8CFFC
:10001000F7CFF6CFF5CFF4CFF3CFF2CFF1CFF0CFCC
:10002000EFCFEECFEDCFECCFEBCF9EC1E9CFE8CF56
:10003000E7CFE6CF1027E80364000A0001000010B4
:100040000001100001001027881301001F0A81031E
:10005000C2175240EAE6BC4001000D4856436F6E9D
:1000600076657274657252326220414444523D2575
:10007000752048563D25750D004D65617375726597
:10008000204D494E20766F6C7461676520000D45E8
:1000900052523A20496E636F727265637420766FB4
:1000A0006C746167650D004D656173757265204DF7
:1000B000415820766F6C7461676520004D656173EF
:1000C000757265204D4944444C4520766F6C7461CF
:1000D00067652000414443203D202575000D565F93
:1000E000544F5F50574D202A2031305E33203D2041
:1000F0002575000D4144435F544F5F56202A20313F
:10010000305E33203D202575000D43414C4942525D
:100110004154494F4E204F4B0D00653D25750D0054
:100120004856203D2025750D004856204F46460D67
:10013000004856204F4E0D004F43523142203D2083
:1001400025750D0001002D4E414E00494E46000020
:100150000100930158000100940144010000F8944B
:10016000EE27EFBBE5BFF8E1A895A4B7A77FA4BF32
:10017000F0936000E09360008DE0A2E0BB27ED9378
:100180008A95E9F780E092E0A0E0B1E0ED93019775
:10019000E9F7E0E5F1E085919591009761F0A5918F
:1001A000B59105901590BF01F00105900D92019752
:1001B000E1F7FB01F0CFE0E0EEBBEFEFEDBFE2E0F7
:1001C000EEBFC0E8D1E05BC1AA935B9AE881E093FF
:1001D000C600B3D3E074E9F3B0D3E064E093C000A9
:1001E0005B980AC0AA93A881AD3021F4ADE0ECDFA2
:1001F000AAE0EADFA881E8DF219608951BD600E097
:1002000010E0A1D23E2EA32D87D3E03069F0A8954F
:10021000AAE0A09FF001A19FF00D8F01E32D90D3E4
:10022000F0970E0F1F1F01C001C0EBCFF8010CD6D5
:100230000895E0E0E5B9E4E0E4B9E0E0E8B9E7B961
:10024000E0E2EBB9EAE2EAB9E0E0E4BDE5BDE6BD33
:10025000E7BDE8BDE3E3E0938000E9E1E0938100DE
:10026000E0E0E0938500E0938400E0938700E09372
:100270008600E7E2E0938900E0E1E0938800E0E0B7
:10028000E0938B00E0938A00E093B600E093B00027
:10029000E093B100E093B200E093B300E093B400C8
:1002A000E0936900EDBBE0936800E0936E00E0939B
:1002B0006F00E0937000E093C000E8E1E093C100BC
:1002C000E6E0E093C200E0E0E093C500EDE4E093F7
:1002D000C400E0E8E0BFE0E0E0937B00E0937F0053
:1002E000E2E0E0937E00EFE8E0937A00E1ECE09357
:1002F0007C00E0E0ECBDE093BC00A895E8E3E0936F
:100300006000E8E2E093600008951CD3E981E09387
:100310008B00E881E0938A002296089513D38AD552
:1003200014D37A168B0610F47A828B820ED3A5151D
:10033000B60510F45A826B820BD3E519F6090BD37C
:100340000ED316D38F01D801E0DFF89414D378943C
:1003500078D524960895F8940ED37894E09192017C
:10036000E030E1F320D308950A921A92FA926A9348
:100370007A938A939A93AA93BA93EA93FA93EFB7EC
:10038000EA9356D5E0917800F09179009F01F90148
:100390000FD317D3C6D4E0938C01F0938D016093F3
:1003A0008E0170938F01A8E8B1E0FAD4EF5FFF4FA0
:1003B0006F4F7F4FFAD4E436A0E0FA07A0E06A0757
:1003C000A0E07A0708F44AC0F3D2E4E6F0E060E087
:1003D00070E0BDD4E0939001F0939101E0E0E093F0
:1003E0008C01E0938D01E0938E01E0938F01E09307
:1003F0008801E0938901E0938A01E0938B01E1E0B9
:10040000E0939201E0919301E03041F1CCD2A3D28C
:10041000DBD2AED2BE2ECF2EE0918B00FE2FE0E0DD
:10042000DF01E0918A008CD2EA0FFB1F8F01B91423
:10043000CA0420F40031E7E21E0708F003C00F5F92
:100440001F4F0AC09B14AC0420F4002400160106C0
:1004500008F002C001501040D80157DFBED2EFD4DF
:100460002496E991EFBFF991E991B991A9919991F8
:10047000899179916991F990199009901895269729
:10048000A0E0B0E0A8D44E2EA1E0B0E0A0D45E2E53
:100490006F2EA3E0B0E09BD47E2E8F2EA5E0B0E0BF
:1004A00092D4A1D2A9E0B0E08ED4A6D2ADE0B0E063
:1004B0008ED49E2EAF2EBDDEA0EDB7E0FDD2EAE5D4
:1004C000F0E0A3D2A5D2AAD2ACD288E007D22A9675
:1004D000A92DBA2D23DF5D9A78947FD2A8952DD2CD
:1004E000E07809F42EC12FD1AE2F1FD21E2F133466
:1004F00071F0113461F0163551F0173541F01834B0
:1005000031F0133521F0173411F0103509F401C022
:10051000E5CF8AD2E42DD90113D2EA17FB0729F0DF
:10052000EDEFF0E0E217F30709F401C0D7CFE12FB8
:1005300007D2E334A0E0FA0709F099C0E0E077D2EF
:10054000A0E0B0E0E2DEE9E7F0E074D2A89556DE84
:10055000AF01042E052A21F04938E3E15E0718F0C7
:100560006ED270D2BBCFA0E1B7E2CFDEE7EAF0E017
:1005700061D2A89543DEEC83FD8366D2309731F0DB
:10058000AC81BD81A938E3E1BE0718F058D25AD238
:10059000A5CFA8E8B3E1B9DEECEBF0E04BD2A8952B
:1005A0002DDEEA83FB83D4D1309749F0CED1A41756
:1005B000B50728F049D2C9D1EA17FB0718F43FD292
:1005C00041D28CCFA895C7DEE883F983E4EDF0E053
:1005D0001CD2BED126D23BD2FA01A1E0B0E00ED4AB
:1005E00033D2A3E0B0E00AD42FD2E41BF50BB3D191
:1005F000A0E0B0E48CE196E44BD3F5D1E09180012A
:10060000F09181016091820170918301A5E0B0E0D9
:10061000EDD3EDEDF0E0F9D1A2D11DD221D298D1E8
:100620009AD1DF01CB01E881F98195D131D3E4D1B1
:10063000E0918401F09185016091860170918701BC
:10064000A9E0B0E0D3D3E3EFF0E0DFD1BDD103D236
:1006500007D2942EA52EE2D1ADE0B0E0CFD3A92DE4
:10066000BA2D5CDEEFD1E9E0F1E0E4D16AC0E1341B
:10067000A0E0FA07B9F4E0E2E31571F4D5D1022E57
:10068000032A21F02D3FE0E03E0708F005C0422E8E
:10069000E22FA0E0B0E0BAD3E5E7F0E0B6D1B8D100
:1006A000D6D14FC0E635A0E0FA0799F4BDD1022EAD
:1006B000032A41F0922EA32EF901ADE0B0E09ED3C3
:1006C000D9012CDEEAE1F1E0A0D1A8D1AAD1BFD1B5
:1006D00038C0E735A0E0FA0739F4E0E2F1E095D15F
:1006E0009DD19FD1B4D12DC0E834A0E0FA0741F4E8
:1006F000EAE1F1E08AD1EB2DFC2D93D1A8D121C004
:10070000E335A0E0FA0729F45D98E9E2F1E092D13F
:1007100018C0E734A0E0FA0729F45D9AE1E3F1E0BC
:1007200089D10FC0E035A0E0FA0759F4E0E07FD1AD
:100730007BD1D901EADDE8E3F1E067D1F90171D1BC
:1007400086D1CCCEFFCFF9D0E078E9F3E091C600B6
:100750000895F8D0AA8146DDA881B981ED91FD9177
:100760003196FE93EE9323960895ECD024975ED3B2
:1007700010E0AA85BB85E0E0F0E0ED93FC93E8890A
:10078000F9893196E88BF98B6FD109F4A1C0E12F7B
:10079000E03031F4353211F411E001C06AD197C074
:1007A000E13081F4353211F464D190C012E020E0E0
:1007B00000E03B3211F42BE28AC0303211F420E227
:1007C00086C002C0E23031F4303319F4006115E024
:1007D0007EC003C0E53009F07AC0E32FE33639F478
:1007E0004FD151D14DD1A481AA9351D16FC0E337DC
:1007F00069F453D154D1AE81BF81ED91AE83BF83F3
:100800003E2FE03011F035D1F6CF60C0E03761F413
:1008100044D145D1EE81FF813196EE83FF8324D10F
:1008200011F027D1F7CF52C0E43611F0E93611F4B8
:10083000016002C0E53719F4E4E3F0E009C0E835EF
:1008400011F4026003C0E83709F040C0EEE3F0E0C5
:10085000EE83FF8300FF0DC020D128D1552322F461
:10086000FA0164D2AF012DE2203011F02A930FD1AA
:1008700002C013D11BD130E3EE81FF819BD2E88708
:10088000F987EE81FF813296EE83FF83E885F98553
:100890004E175F0730F03F5FA885B9854A1B5B0B99
:1008A000F5CF04FD06C0313320F4A885B985119732
:1008B00049F400613A3328F001FF02C0395F01C0FA
:1008C000395DD7D0A885B9851297A8F610E057CF23
:1008D000AA85BB8561D2B1D262960895FF92F82EA7
:1008E0002697A8D2DE01149618D28D01E0E0EC83A1
:1008F000ED83EE83EF83DE0118960FD24DD285D0C3
:100900001A930A93E9EAF3E080D0DE0118962DDF0E
:1009100098D22896FF900895AA93E1E0F991F033D8
:1009200010F0FA3308F0EE270895AA93E991E13622
:1009300018F0EB3708F4E0520895E091C0000895F4
:10094000F0E00895BA93AA930895AA81BB8108950F
:10095000EA81FB810895662777271ED10895A0912B
:100960008001B0918101809182019091830108956D
:1009700041D1D9D00895E0E0E0938C01E0938D015E
:10098000E0938E01E0938F01E0938801E093890169
:10099000E0938A01E0938B01E0939001E093910151
:1009A000E09392010895E0919001F09191010895F2
:1009B000A0918C01B0918D0180918E0190918F0159
:1009C0000895662777270895A0918401B091850145
:1009D00080918601909187010895E0917A00E0640A
:1009E000E0937A000895E0938001F0938101609391
:1009F0008201709383010895E0938401F09385014F
:100A000060938601709387010895FA93EA9308959D
:100A1000E42DFF2766277727D1D10895E92DFA2DF8
:100A20000895CFDFCBD10895E9DB9F010895E093CE
:100A300093010895EADF80E051DF22960895EEE801
:100A4000F0E0F8CFE1E0F3CFEC81FD81089584E0A0
:100A500045DF26960895E0E0F0E06AE774E488CF89
:100A6000B0DFAFDFABD1F3CF3197E4913E2FE03071
:100A700008953A93AB85BC85ED85FE85099508956B
:100A8000EE85FF8508953497EE87FF870895AB853F
:100A9000BC85ED85FE8509950895F2DFF4CFAE851E
:100AA000BF85149679D1EE83FF830895AE85BF8507
:100AB00014964D915C910895109639F088EB9BE067
:100AC0000197F1F7A8951197C9F70895552342F4B6
:100AD000503811F4E0FF04C03196691F791F6BF0A4
:100AE00050E8572711F45F9373C05F3F31F0660FF2
:100AF000000C57956795752F08955F9300200AF0B5
:100B000073C06CC050E8192E1522880F991F9527C5
:100B1000550F879550E8072E0522660F771F75271A
:100B2000550F67950895689401C0E8945F93F2DFCC
:100B3000703818F07F3F08F44BC056E1571BAAF4F9
:100B4000519558300EF4593030F0EFEFFFEF6FEF62
:100B50007FE777F91AC077275523B9F0EE0FFF1F0B
:100B6000661F771F5A95D1F710C07727583028F0A5
:100B7000EF2FF62F672F5850F9CF552331F0769588
:100B80006795F795E7955A95D1F700200AF4D2D0EA
:100B90005F910895689401C0E89430976040704078
:100BA000B1F0002426F0772312F40094C3D0172E5E
:100BB0007EE1112032F07A95EE0FFF1F661F111CA7
:100BC000F9CFEF2FF62F612D5F938ADF5F910895A4
:100BD000EE27FF27662777275F910895EFEFFFEF56
:100BE0006FE77FEF5F910895EFEFFFEF6FE77FE72C
:100BF0005F9108955F9386DF703851F3903841F329
:100C000001240894791F23F41CF300203AF3ECCF5D
:100C10000F921F932F933F934F93112722279927CA
:100C2000689FA0018F9F302D410D591F6B9F300D84
:100C3000411D591F8E9F27D0BF9F25D06A9F23D06B
:100C4000BE9F1DD0AF9F1BD0AE9F110D291F391F16
:100C5000491F591FE32FF42F652F522F4F913F91BA
:100C60002F911F910F9066232AF0550FEE1FFF1F43
:100C7000661F02C073954BF229DF5F910895100D36
:100C8000211D391F02C0200D311D491F591F089514
:100C90005F9338DF703821F411200AF49FCFA4CF7E
:100CA000903809F495CF01240894970B1BF4D4F3E2
:100CB0000020F3CF792F1F932F933F934F9311244D
:100CC0001127222733274427552790E2AE17BF0765
:100CD0008607410730F0AE1BBF0B860B410B089413
:100CE00001C08894551F221F331F111CAA1FBB1F50
:100CF000881F441F9A9551F7F901612D4F913F913B
:100D00002F911F91662332F0550FEE1FFF1F661FB4
:100D10007A9543F2DBDE5F9108950024AF0DB01D9C
:100D20000895EA0FFB1F681F791F0895F195E1955B
:100D3000F0400895F09560957095E195FF4F6F4FE5
:100D40007F4F08956F2F660F660B762F08953F93A0
:100D50004F935F93002411244427552730E2AA0FB4
:100D6000BB1F881F991F001C111C441F551F0E1A02
:100D70001F0A460B570B28F40E0E1F1E461F571F47
:100D800001C0A1603A9559F7FD01BC01D001CA012B
:100D90005F914F913F910895ED91FC9111970895C6
:100DA000ED91FD916D917D9108957E936E93FE93EB
:100DB000EE9308950590F491E02D08957A936A9347
:100DC000FA93EA930895129602D0BF0112971196F2
:100DD00002D0FE2F1197F999FECFFF93FFB7F89439
:100DE000A1BDF89AE0B5FFBFFF91089507D0129614
:100DF0000F01FB0103D0F0011297089507D011965F
:100E0000EF93EF2F03D0EF9111970895F99B02C054
:100E1000A895FCCF9FB7F894A1BDF89A80B5E817C4
:100E200019F0E0BDFA9AF99A9FBF08955A934A9330
:100E30003A932A931A930A9308955D814C813B81DA
:100E40002A81198108810895099119910895FFFF58
:100E5000FFFFFFFFFFFFFFFFFFFFFFFFFFFFFFFFA2
:100E6000FFFFFFFFFFFFFFFFFFFFFFFFFFFFFFFF92
:100E7000FFFFFFFFFFFFFFFFFFFFFFFFFFFFFFFF82
:100E8000FFFFFFFFFFFFFFFFFFFFFFFFFFFFFFFF72
:100E9000FFFFFFFFFFFFFFFFFFFFFFFFFFFFFFFF62
:100EA000FFFFFFFFFFFFFFFFFFFFFFFFFFFFFFFF52
:100EB000FFFFFFFFFFFFFFFFFFFFFFFFFFFFFFFF42
:100EC000FFFFFFFFFFFFFFFFFFFFFFFFFFFFFFFF32
:100ED000FFFFFFFFFFFFFFFFFFFFFFFFFFFFFFFF22
:100EE000FFFFFFFFFFFFFFFFFFFFFFFFFFFFFFFF12
:100EF000FFFFFFFFFFFFFFFFFFFFFFFFFFFFFFFF02
:100F0000FFFFFFFFFFFFFFFFFFFFFFFFFFFFFFFFF1
:100F1000FFFFFFFFFFFFFFFFFFFFFFFFFFFFFFFFE1
:100F2000FFFFFFFFFFFFFFFFFFFFFFFFFFFFFFFFD1
:100F3000FFFFFFFFFFFFFFFFFFFFFFFFFFFFFFFFC1
:100F4000FFFFFFFFFFFFFFFFFFFFFFFFFFFFFFFFB1
:100F5000FFFFFFFFFFFFFFFFFFFFFFFFFFFFFFFFA1
:100F6000FFFFFFFFFFFFFFFFFFFFFFFFFFFFFFFF91
:100F7000FFFFFFFFFFFFFFFFFFFFFFFFFFFFFFFF81
:100F8000FFFFFFFFFFFFFFFFFFFFFFFFFFFFFFFF71
:100F9000FFFFFFFFFFFFFFFFFFFFFFFFFFFFFFFF61
:100FA000FFFFFFFFFFFFFFFFFFFFFFFFFFFFFFFF51
:100FB000FFFFFFFFFFFFFFFFFFFFFFFFFFFFFFFF41
:100FC000FFFFFFFFFFFFFFFFFFFFFFFFFFFFFFFF31
:100FD000FFFFFFFFFFFFFFFFFFFFFFFFFFFFFFFF21
:100FE000FFFFFFFFFFFFFFFFFFFFFFFFFFFFFFFF11
:100FF000FFFFFFFFFFFFFFFFFFFFFFFFFFFFFFFF01
:00000001FF
